:020000020000FC
:1000000003C018953EC0189503E313E320E030E0E9
:100010004FEFEFE0E7BBE1BBE0EFE8BBE2BBE5E0C1
:10002000E3BFE2E0E9BF7894E02FEF70E423E06FF4
:10003000E8BBE12FEF70E423E06FE2BBE6B320956D
:100040002E2320712E2F59F0B59B000FB5990695E0
:1000500004FB00F903FB07F9E0E0E2BF4FEFE0B378
:1000600030953E2330713E2F59F0859B110F8599B5
:10007000169514FB10F913FB17F9E0E0E2BF4FEF00
:0E008000D3CFCFB74095DFEFD2BFCFBF1895DB
:00000001FF
